:060000000A128A110C280F
:10000800FE000308F4000A08F5000A128A15BC2E3F
:100018000A128A11C12F00308A000408840A820754
:100028000034083409340A340B340C340D340E34DB
:100038000F340734063405340434033402340134ED
:100048000034C900D300AF01B001B101B201D4013D
:100058003C28AF01AF0A4C28B001B00A4C28B101C6
:10006800B10A4C28B201B20A4C28D401D40A4C284F
:100078004908013A03192D28033A03193028013A8F
:1000880003193328073A03193628013A031939287E
:10009800831603178C184C28083083128D0003131D
:1000A8005308A6230A128A1103188B178C185A288A
:1000B800093083128D0003132F08A6230A128A1110
:1000C80003188B178C1866280A3083128D000313C7
:1000D8003008A6230A128A1103188B178C18722865
:1000E8000B3083128D0003133108A6230A128A11DC
:1000F80003188B178C187E280C3083128D0003137D
:100108003208A6230A128A1103188B178C188A281A
:100118000D3083128D0003135408A6230A128A1186
:1001280003188B17BF2AD508031D9D28D501D50AAA
:100138009E28D501AB01AB0ABF2AC900D801BA0174
:10014800B501A601B328D801D80AC028BA01BA0A4D
:10015800C028B501B50AC028A601A60AC0284908C2
:10016800013A0319A728033A0319AA28013A0319DF
:10017800AD28073A0319B028B7238C18C028831272
:100188008D0103135808A6230A128A1103188B1726
:100198008C18CC28013083128D0003133A08A6234B
:1001A8000A128A1103188B178C18D8280230831268
:1001B8008D0003133508A6230A128A1103188B171A
:1001C8008C18E428033083128D0003132608A62315
:1001D8000A128A1103188B17BF2AD608031DF7289D
:1001E800D601D60AF828D601BF220A128A11B723E7
:1001F8008C18FB28073083128D0003135608A6239A
:1002080003188B170800D208031D0D29D201D20A42
:100218000E29D2010330AB00BF220A128A11B7237C
:100228008C181329063083128D0003135208A62355
:1002380003188B170800D708031D2529D701D70AEB
:100248002629D7010230AB00BF220A128A11B72330
:100258008C182B29053083128D0003135708A62309
:1002680003188B170800580B5D29BB03FB303B02B2
:100278000318BB010630C600C7014F30CE003B084B
:100288004E02C800C901031CC90361230A128A115E
:10029800460831220A128A11B7238C1850290E30C9
:1002A80083128D0003133B08A6230A128A11031830
:1002B8008B17BA233A0B7729B903FB303902031895
:1002C800B90139080F3C31220A128A11B7238C1858
:1002D8006A290F3083128D0003133908A6230A12E6
:1002E8008A1103188B17BA23350B9129B403FB30F5
:1002F80034020318B40134080F3C31220A128A115F
:10030800B7238C188429103083128D000313340806
:10031800A6230A128A1103188B17BA23260BAB29B6
:10032800A503FB3025020318A50125080F3C31223F
:100338000A128A11B7238C189E29113083128D0056
:1003480003132508A6230A128A1103188B17FF30F6
:10035800BA23A200A3000800580BD829BB0A5030C2
:100368003B02031CB9294F30BB000630C600C70149
:100378004F30CE003B084E02C800C901031CC90318
:1003880061230A128A11460831220A128A11B723F8
:100398008C18CB290E3083128D0003133B08A6233B
:1003A8000A128A1103188B17BA233A0BF429B90ACF
:1003B80010303902031CE2290F30B90039080F3C0C
:1003C80031220A128A11B7238C18E7290F308312B9
:1003D8008D0003133908A6230A128A1103188B17F4
:1003E800BA23350B102AB40A10303402031CFE2934
:1003F8000F30B40034080F3C31220A128A11B72397
:100408008C18032A103083128D0003133408A62396
:100418000A128A1103188B17BA23260B2C2AA50A4D
:1004280010302502031C1A2A0F30A50025080F3C9E
:1004380031220A128A11B7238C181F2A113083120D
:100448008D0003132508A6230A128A1103188B1797
:10045800FF30BA23A200A3000800BA23C800480846
:1004680003193A2AC601C701C70A3C2AC601C701AF
:1004780008303E230A128A1102304802C601C60A11
:10048800C7010318C70A08303E230A128A1103302D
:1004980048020330C600C7010318C70A07303E23C5
:1004A8000A128A1104304802C601C60AC701031895
:1004B800C70A07303E230A128A110530480206305F
:1004C800C600C7010318C70A05303E230A128A115D
:1004D800063048020730C600C7010318C70A0530AE
:1004E8003E230A128A1107304802C601C60AC7010C
:1004F8000318C70A09303E230A128A110830480235
:10050800C601C7010318C70A09303E230A128A1117
:10051800093048020330C600C7010318C70A05306E
:100528003E230A128A110A3048020230C600C70167
:100538000318C70A05303E230A128A110B304802F5
:10054800C601C7010318C70A05303E230A128A11DB
:100558000C304802C601C60AC7010318C70A05308D
:100568003E230A128A110D3048020530C600C70121
:100578000318C70A3E2B003031220A128A110330B1
:10058800C6002C08C70008303E230A128A112C0B1B
:10059800D12A0230C600C701D52A0230C600C701D9
:1005A800C70A08303E230A128A112C0B0800C6011C
:1005B8005808C70008303E230A128A11C601C60A25
:1005C8003A08C70008303E230A128A110330C600D1
:1005D8003508C70007303E230A128A11C601C60A29
:1005E8002608C70007303E230A128A110630C600C3
:1005F8005508C70005303E230A128A110730C60085
:100608005708C70005303E230A128A11C601C60AD8
:100618005208C70009303E230A128A11C60156083B
:10062800C70009303E230A128A110330C6002F087A
:10063800C70005303E230A128A110230C60030086E
:10064800C70005303E230A128A11C6013108C700C7
:1006580005303E230A128A11C601C60A3208C700AD
:1006680005303E230A128A110530C6005408C70017
:1006780005303E2BF70047080319512B77088400F3
:100688000130F600460A4A2B0310F60DFF3E031D03
:10069800482B76088313800408007708840001300B
:1006A800F600460A592B0310F60DFF3E031D572B83
:1006B8007608FF3A831380050800CB01C71F6B2B10
:1006C800C609C709C60A0319C70ACB01CB0AC91F3D
:1006D800742BC809C909C80A0319C90A0130CB060D
:1006E800CC01CD01470846040319992BCA01CA0A4F
:1006F800C71B822B0310C60DC70D7B2B0310CC0D17
:10070800CD0D47084902031D8B2B46084802031CE0
:10071800952B4608C8024708031CC903C9024C1494
:100728000310C70CC60CCA0B822B4B080319A12B4C
:10073800CC09CD09CC0A0319CD0A4D08C7004C08CD
:10074800C600080003178C003F3083168C05031081
:100758008B1B03148B130C1555308D00AA308D009C
:100768008C140C1108008316031708008312031356
:100778000800FF30CF00D0000130CF020030031C4A
:10078800D003D0024F0A0319500A031DC02B0A12C6
:100798008A1190270A128A110A128A15F6250A1256
:1007A8008A11D501D50AAC010A128A11BF220A1290
:1007B8008A110A128A11B2260A128A110A128A1199
:1007C8008B260A128A110A128A15F6250A128A112C
:1007D8008B17330803198A2C2C0B722C4A2C0130E6
:1007E8000A128A11A1200A128A11722C02300A12E6
:1007F8008A11A1200A128A11722C03300A128A1156
:10080800A1200A128A11722C04300A128A11A1201E
:100818000A128A11722C0A128A1197200A128A1156
:10082800722C0A128A111F210A128A11722C0A12BA
:100838008A1107210A128A11722C0A128A11F120D0
:100848000A128A11722C01300A128A1125200A1202
:100858008A11722C02300A128A1125200A128A1172
:10086800722C03300A128A1125200A128A11722C5E
:1008780004300A128A1125200A128A11722C0530B6
:100888000A128A1125200A128A11722C3308013A99
:100898000319F32B033A0319FA2B013A0319012C14
:1008A800073A0319082C013A03190F2C033A0319C4
:1008B800152C013A03191B2C0F3A0319212C013A64
:1008C8000319272C033A03192E2C013A0319352C46
:1008D800073A03193C2C013A0319432C83120313DA
:1008E80033080E3A031D7D2C0A128A11D4250A12E8
:1008F8008A110A128A11E9250A128A110A128A1122
:100908004D260A128A11B308031D872C280BA42C24
:100918002C0BA42C8F018E01A801AA08031D9A2C68
:100928000A128A11B0210A128A119F2C0A128A11FE
:1009380037210A128A110A128A11E9250A128A1124
:10094800A801230822040319B82C0130A2020030A0
:10095800031CA303A30222032304031DB82C0A12B9
:100968008A11BF220A128A11210820040319C22CF5
:100978000130A0020030031CA103A10224080319BE
:10098800ED2B24080C3A031DD22C21082004031D4A
:10099800D22C0A128A11D4250A128A112C0BC42DC2
:1009A80024082B3A031DDE2C01300A128A11A120DB
:1009B8000A128A1124082C3A031DE82C02300A1264
:1009C8008A11A1200A128A1124082D3A031DF22C3B
:1009D80003300A128A11A1200A128A1124082E3A19
:1009E800031DFC2C04300A128A11A1200A128A1154
:1009F80024080D3A031D092D21082004031D092D83
:100A08000A128A1197200A128A112408073A031D2C
:100A1800162D21082004031D162D0A128A111F21E4
:100A28000A128A11831203132408083A031D252D7C
:100A380021082004031D252D0A128A1107210A12F4
:100A48008A11831203132408093A031D342D21083F
:100A58002004031D342D0A128A11F1200A128A116A
:100A6800831203132408103A031D5C2D2108200467
:100A7800031D5C2D350B482DB501A601A60A0A12E7
:100A88008A11BF220A128A113A0B522DBA01B501F6
:100A9800B50A0A128A11BF220A128A11580B5C2D54
:100AA800D801BA01BA0A0A128A11BF220A128A1197
:100AB8002408113A031D822D21082004031D822DCC
:100AC8003A0B6E2DBA01D801D80A0A128A11BF2230
:100AD8000A128A11350B782DB501BA01BA0A0A1221
:100AE8008A11BF220A128A11260B822DA601B5018E
:100AF800B50A0A128A11BF220A128A11240B8A2DFA
:100B080001300A128A1125200A128A112408023A91
:100B1800031D942D02300A128A1125200A128A1107
:100B28002408033A031D9E2D03300A128A1125203A
:100B38000A128A112408043A031DA82D04300A1247
:100B48008A1125200A128A112408053A031DB22D9C
:100B580005300A128A1125200A128A112408153A2A
:100B6800031DBB2D0A128A11B0210A128A1124080A
:100B7800163A031DC42D0A128A1137210A128A1146
:100B8800FF30A0000F30A100A4010A128A11E92544
:100B98000A128A110A128A114D260A128A11ED2B9D
:100BA800AC08031DDB2DAC01AC0AD501DE2DAC0170
:100BB800D501D50AAB01AB0A0A128A11BF220A1263
:100BC8008A11E9250A128A114D2E37270A128A112D
:100BD800883017270A128A112B080319092E550B7A
:100BE800F72DD115F82DD111D208031DFD2D511562
:100BF800FE2D5111D708031D032ED114042ED11038
:100C0800AB01510817270A128A11580B222ECB0163
:100C18003B08CC000A304C02031C162ECB0AF630D7
:100C2800CC070E2EE030CB07D030CC074C08172766
:100C38000A128A114B0817270A128A113A0B302E0A
:100C48003908013E84000A128A110F200A128A11FB
:100C5800B03E17270A128A11350B3E2E3408013E82
:100C680084000A128A110F200A128A11A03E17273F
:100C78000A128A11260B4C2E2508013E84000A12FE
:100C88008A110F200A128A11903E17270A128A1118
:100C9800532F37270A128A11943017270A128A11FC
:100CA8006E2ECB3017270A128A117E2ECA301727CC
:100CB8000A128A117E2EC93017270A128A117E2E2F
:100CC800C83017270A128A117E2EC73017270A1232
:100CD8008A117E2E5308013A0319552E033A031937
:100CE8005A2E013A03195F2E073A0319642E013A66
:100CF8000319692E560B822ED030832ED130172738
:100D08000A128A11913017270A128A11532F37278E
:100D18000A128A11943017270A128A11F0301727FD
:100D28000A128A11F23017270A128A11F43017278B
:100D38000A128A11F63017270A128A11F830172773
:100D48000A128A11FA3017270A128A11FE30172759
:100D58000A128A1153270A128A114D2E37270A12AE
:100D68008A11883017270A128A11FF3017270A12AA
:100D78008A1153270A128A1137270A128A118830D2
:100D880017270A128A11C73017270A128A11532700
:100D98000A128A1137270A128A11883017270A126D
:100DA8008A11703017270A128A1153270A128A11DA
:100DB800AB01AB0AD801D80ABA01BA0AB501B50A1B
:100DC800A601A60AE9250A128A11BA01B501A601E7
:100DD800B801B701B601A701AE01AD0137270A1264
:100DE8008A11883017270A128A112D08103E1727F2
:100DF8000A128A112E08203E17270A128A1127087C
:100E0800303E17270A128A113608403E17270A1261
:100E18008A113708503E17270A128A11603017279F
:100E28000A128A11532FC9000830CA00CA080319C8
:100E3800352FCA034908C8004A0A242F0310C80CD2
:100E4800FF3E031D222F4808C7000130C7050230A6
:100E5800C600073061270A128A1184270A128A11EC
:100E68001A2F0000842F0230C600C701C70A0730B6
:100E780061270A128A11C601C701C70A073061270C
:100E88000A128A1100000230C600C7010730612724
:100E98000A128A110000C601C7010730612FC60176
:100EA800C701C70A073061270A128A1100000230F9
:100EB800C600C701C70A0730612FF70047080319A2
:100EC800742F770884000130F600460A6D2F03104E
:100ED800F60DFF3E031D6B2F760883138004080070
:100EE800770884000130F600460A7C2F0310F60DBF
:100EF800FF3E031D7A2F7608FF3A8313800508000A
:100F0800C601C701C70A073061270A128A11000003
:100F1800C601C7010730612F8B0183160F178F1683
:100F28000F12031788018901103003138500F6306A
:100F3800860087018801890183128501860187015E
:100F4800880189018316811395000B1783121012EB
:100F580090129011901010148F018E0183160C14AA
:100F6800C03096008B150B10811601168115FF30C5
:100F7800831281008B160B11080083132030840024
:100F88003C300A128A11D8277030D1000130D200C3
:100F98000530D3000130D400D500D600D700D800E2
:100FA80083010A128A11BD2B64008001840A040699
:080FB800031900340406D92FCF
:101BEC0003178D013F3083168C050C1483120C08DF
:101BFC000313D800013003178D003F3083168C057A
:101C0C000C1483120C080313BA00023003178D0056
:101C1C003F3083168C050C1483120C080313B5008B
:101C2C00033003178D003F3083168C050C14831280
:101C3C000C080313A600043003178D003F308316E5
:101C4C008C050C1483120C080313D50005300317F4
:101C5C008D003F3083168C050C1483120C08031373
:101C6C00D700063003178D003F3083168C050C14FB
:101C7C0083120C080313D200073003178D003F307A
:101C8C0083168C050C1483120C080313D600083031
:101C9C0003178D003F3083168C050C1483120C082F
:101CAC000313D300093003178D003F3083168C05C6
:101CBC000C1483120C080313AF000A3003178D00A9
:101CCC003F3083168C050C1483120C080313B000E0
:101CDC000B3003178D003F3083168C050C148312C8
:101CEC000C080313B1000C3003178D003F30831622
:101CFC008C050C1483120C080313B2000D3003175F
:101D0C008D003F3083168C050C1483120C080313C2
:101D1C00D4000E3003178D003F3083168C050C1445
:101D2C0083120C080313BB000F3003178D003F30D8
:101D3C0083168C050C1483120C080313B900103095
:101D4C0003178D003F3083168C050C1483120C087E
:101D5C000313B400113003178D003F3083168C052C
:101D6C000C1483120C080313A500080001300B1C83
:101D7C0000398B1D003900380319E02E0B10003090
:101D8C0083120313061B0130BC000030861B01308C
:101D9C00C30029060319DE2E3C030319DE2E430370
:101DAC000319DB2EAA01AA0ADC2EAA01A801A80A93
:101DBC004308A9000130831203130C1C003983164D
:101DCC000C1C003900380319A02F83120C107F3023
:101DDC008F00FF308E00B301081688170614861585
:101DEC008712C401C40AC501FA270A128A150319FD
:101DFC00450A031DFA2E8618052FB301B30A061ADD
:101E0C00092F0930B3008716C401C40AC501FA278B
:101E1C000A128A150319450A031D0D2F0812C40155
:101E2C00C40AC501FA270A128A150319450A031DAB
:101E3C00182F8618232F0230B3000619272F0630CF
:101E4C00B300061A2B2F0A30B3000816C401C40ABB
:101E5C00C501FA270A128A150319450A031D2F2FEB
:101E6C008813C401C40AC501FA270A128A1503197A
:101E7C00450A031D3A2F8618452F0330B300061967
:101E8C00492F0730B300061A4D2F0B30B3008817BB
:101E9C00C401C40AC501FA270A128A150319450A96
:101EAC00031D512F0610C401C40AC501FA270A12DA
:101EBC008A150319450A031D5C2F8618672F0430F9
:101ECC00B30006196B2F0830B300061A6F2F0C30B5
:101EDC00B3000614C401C40AC501FA270A128A15F4
:101EEC000319450A031D732F8611C401C40AC501C9
:101EFC00FA270A128A150319450A031D7E2F861824
:101F0C00892F0530B300061A8D2F0D30B3008615BE
:101F1C00C401C40AC5010130C4020030031CC5034E
:101F2C00C502440A0319450A031D912F861AA02FD6
:101F3C000E30B30001300B1D00398B1E00390038F8
:101F4C000319F32F8312BE01BE0ABF01C001A030DA
:101F5C00C100C2010130C102031CC203410A0319B2
:101F6C00420A031DB02F0310051A03140030031886
:101F7C000130F000F1013F08F3003E08F2000310BD
:101F8C00F20DF30D70087207BE0071080318710A88
:101F9C007307BF000030051A0130BD003230C1009C
:101FAC00C201420841040319E72F0130C10200307D
:101FBC00031CC203051A01303D060319D72FC101BA
:101FCC00D62FC00A0D304002031CAD2FFF3081000C
:101FDC000B113E08A4003F30A40575088A00740854
:101FEC008300FE0E7E0E09000130C402031CC503E3
:041FFC00440A08008B
:02400E00C423C9
:1042000001000000000000000000010001000100AA
:10421000050000000000000000000100140008007C
:1042200008000800FF00FF00FF00FF00FF00FF0084
:00000001FF
